BL51 BANKED LINKER/LOCATER V6.22                                                        04/19/2018  15:18:06  PAGE 1


BL51 BANKED LINKER/LOCATER V6.22, INVOKED BY:
D:\KEIL_51\C51\BIN\BL51.EXE STARTUP.obj, main.obj, oled.obj TO OLED RAMSIZE (256)


MEMORY MODEL: SMALL


INPUT MODULES INCLUDED:
  STARTUP.obj (?C_STARTUP)
  main.obj (MAIN)
  oled.obj (OLED)
  D:\KEIL_51\C51\LIB\C51S.LIB (?C?CLDOPTR)
  D:\KEIL_51\C51\LIB\C51S.LIB (?C?IMUL)
  D:\KEIL_51\C51\LIB\C51S.LIB (?C?UIDIV)
  D:\KEIL_51\C51\LIB\C51S.LIB (?C?OFFXADD)


LINK MAP OF MODULE:  OLED (?C_STARTUP)


            TYPE    BASE      LENGTH    RELOCATION   SEGMENT NAME
            -----------------------------------------------------

            * * * * * * *   D A T A   M E M O R Y   * * * * * * *
            REG     0000H     0008H     ABSOLUTE     "REG BANK 0"
            DATA    0008H     000DH     UNIT         _DATA_GROUP_
            DATA    0015H     0009H     UNIT         ?DT?_OLED_SHOWNUM?OLED
            DATA    001EH     0001H     UNIT         ?DT?_OLED_POW?OLED
            IDATA   001FH     0001H     UNIT         ?STACK

            * * * * * * *   C O D E   M E M O R Y   * * * * * * *
            CODE    0000H     0003H     ABSOLUTE     
            CODE    0003H     3232H     UNIT         ?CO?MAIN
            CODE    3235H     09D8H     UNIT         ?CO?OLED
            CODE    3C0DH     0161H     UNIT         ?PR?_OLED_SHOWCHAR?OLED
            CODE    3D6EH     0124H     UNIT         ?PR?_OLED_SHOWCHINESE?OLED
            CODE    3E92H     00B8H     UNIT         ?PR?MAIN?MAIN
            CODE    3F4AH     00A0H     UNIT         ?PR?INITIAL_SSD1327?OLED
            CODE    3FEAH     00A0H     UNIT         ?C?LIB_CODE
            CODE    408AH     007EH     UNIT         ?PR?_OLED_DRAWBMP?OLED
            CODE    4108H     0075H     UNIT         ?PR?_OLED_SHOWNUM?OLED
            CODE    417DH     0031H     UNIT         ?PR?_OLED_SHOWSTRING?OLED
            CODE    41AEH     002AH     UNIT         ?PR?RAINBOW?OLED
            CODE    41D8H     0026H     UNIT         ?PR?_WRITE_IIC_BYTE?OLED
            CODE    41FEH     0022H     UNIT         ?PR?_CLEARLED?OLED
            CODE    4220H     001FH     UNIT         ?PR?_DELAY?OLED
            CODE    423FH     0018H     UNIT         ?PR?_OLED_POW?OLED
            CODE    4257H     0017H     UNIT         ?PR?_COLUMN_ADDRESS?OLED
            CODE    426EH     0013H     UNIT         ?PR?_WRITE_REGISTER?OLED
            CODE    4281H     0013H     UNIT         ?PR?_ROW_ADDRESS?OLED
            CODE    4294H     0013H     UNIT         ?PR?_SET_COLUME_ADDRESS?OLED
            CODE    42A7H     0013H     UNIT         ?PR?_SET_ROW_ADDRESS?OLED
            CODE    42BAH     0010H     UNIT         ?PR?IIC_WAIT_ACK?OLED
            CODE    42CAH     000EH     UNIT         ?PR?_WRITE_PARAMETER?OLED
            CODE    42D8H     000CH     UNIT         ?C_C51STARTUP
            CODE    42E4H     000AH     UNIT         ?PR?OPEN_DC_POWER?OLED
            CODE    42EEH     000AH     UNIT         ?PR?OFF_DC_POWER?OLED
            CODE    42F8H     0009H     UNIT         ?PR?IIC_START?OLED
BL51 BANKED LINKER/LOCATER V6.22                                                      04/19/2018  15:18:06  PAGE 2


            CODE    4301H     0007H     UNIT         ?PR?IIC_STOP?OLED



OVERLAY MAP OF MODULE:   OLED (?C_STARTUP)


SEGMENT                                DATA_GROUP 
  +--> CALLED SEGMENT                START    LENGTH
----------------------------------------------------
?C_C51STARTUP                        -----    -----
  +--> ?PR?MAIN?MAIN

?PR?MAIN?MAIN                        0008H    0001H
  +--> ?PR?INITIAL_SSD1327?OLED
  +--> ?PR?_CLEARLED?OLED
  +--> ?PR?OPEN_DC_POWER?OLED
  +--> ?PR?_OLED_SHOWCHINESE?OLED
  +--> ?CO?MAIN
  +--> ?PR?_OLED_SHOWSTRING?OLED
  +--> ?PR?_OLED_DRAWBMP?OLED
  +--> ?PR?_DELAY?OLED
  +--> ?PR?RAINBOW?OLED

?PR?INITIAL_SSD1327?OLED             -----    -----
  +--> ?PR?_DELAY?OLED
  +--> ?PR?_WRITE_REGISTER?OLED

?PR?_WRITE_REGISTER?OLED             -----    -----
  +--> ?PR?_WRITE_IIC_BYTE?OLED
  +--> ?PR?IIC_WAIT_ACK?OLED
  +--> ?PR?IIC_STOP?OLED

?PR?_WRITE_IIC_BYTE?OLED             -----    -----
  +--> ?PR?IIC_START?OLED

?PR?IIC_WAIT_ACK?OLED                -----    -----
  +--> ?PR?_WRITE_IIC_BYTE?OLED

?PR?_CLEARLED?OLED                   0009H    0001H
  +--> ?PR?_SET_COLUME_ADDRESS?OLED
  +--> ?PR?_SET_ROW_ADDRESS?OLED
  +--> ?PR?_WRITE_PARAMETER?OLED

?PR?_SET_COLUME_ADDRESS?OLED         -----    -----
  +--> ?PR?_WRITE_REGISTER?OLED

?PR?_SET_ROW_ADDRESS?OLED            -----    -----
  +--> ?PR?_WRITE_REGISTER?OLED

?PR?_WRITE_PARAMETER?OLED            -----    -----
  +--> ?PR?_WRITE_IIC_BYTE?OLED
  +--> ?PR?IIC_WAIT_ACK?OLED
  +--> ?PR?IIC_STOP?OLED

?PR?OPEN_DC_POWER?OLED               -----    -----
  +--> ?PR?_WRITE_REGISTER?OLED
BL51 BANKED LINKER/LOCATER V6.22                                                      04/19/2018  15:18:06  PAGE 3



?PR?_OLED_SHOWCHINESE?OLED           0009H    0007H
  +--> ?PR?_SET_COLUME_ADDRESS?OLED
  +--> ?PR?_SET_ROW_ADDRESS?OLED
  +--> ?CO?OLED
  +--> ?PR?_WRITE_PARAMETER?OLED

?PR?_OLED_SHOWSTRING?OLED            0009H    0006H
  +--> ?PR?_OLED_SHOWCHAR?OLED

?PR?_OLED_SHOWCHAR?OLED              000FH    0006H
  +--> ?PR?_SET_COLUME_ADDRESS?OLED
  +--> ?PR?_SET_ROW_ADDRESS?OLED
  +--> ?CO?OLED
  +--> ?PR?_WRITE_PARAMETER?OLED

?PR?_OLED_DRAWBMP?OLED               0009H    000BH
  +--> ?PR?_SET_COLUME_ADDRESS?OLED
  +--> ?PR?_SET_ROW_ADDRESS?OLED
  +--> ?PR?_WRITE_PARAMETER?OLED

?PR?RAINBOW?OLED                     -----    -----
  +--> ?PR?_SET_COLUME_ADDRESS?OLED
  +--> ?PR?_SET_ROW_ADDRESS?OLED
  +--> ?PR?_WRITE_PARAMETER?OLED



SYMBOL TABLE OF MODULE:  OLED (?C_STARTUP)

  VALUE           TYPE          NAME
  ----------------------------------

  -------         MODULE        ?C_STARTUP
  C:42D8H         SEGMENT       ?C_C51STARTUP
  I:001FH         SEGMENT       ?STACK
  C:0000H         PUBLIC        ?C_STARTUP
  D:00E0H         SYMBOL        ACC
  D:00F0H         SYMBOL        B
  D:0083H         SYMBOL        DPH
  D:0082H         SYMBOL        DPL
  N:0000H         SYMBOL        IBPSTACK
  N:0100H         SYMBOL        IBPSTACKTOP
  N:0080H         SYMBOL        IDATALEN
  C:42DBH         SYMBOL        IDATALOOP
  N:0000H         SYMBOL        PBPSTACK
  N:0100H         SYMBOL        PBPSTACKTOP
  N:0000H         SYMBOL        PDATALEN
  N:0000H         SYMBOL        PDATASTART
  N:0000H         SYMBOL        PPAGE
  N:0000H         SYMBOL        PPAGEENABLE
  D:00A0H         SYMBOL        PPAGE_SFR
  D:0081H         SYMBOL        SP
  C:42D8H         SYMBOL        STARTUP1
  N:0000H         SYMBOL        XBPSTACK
  N:0000H         SYMBOL        XBPSTACKTOP
  N:0000H         SYMBOL        XDATALEN
BL51 BANKED LINKER/LOCATER V6.22                                                      04/19/2018  15:18:06  PAGE 4


  N:0000H         SYMBOL        XDATASTART
  C:0000H         LINE#         126
  C:42D8H         LINE#         133
  C:42DAH         LINE#         134
  C:42DBH         LINE#         135
  C:42DCH         LINE#         136
  C:42DEH         LINE#         185
  C:42E1H         LINE#         196
  -------         ENDMOD        ?C_STARTUP

  -------         MODULE        MAIN
  C:0000H         SYMBOL        _ICE_DUMMY_
  D:0090H         PUBLIC        P1
  C:1235H         PUBLIC        BMP2
  C:3E92H         PUBLIC        main
  C:0035H         PUBLIC        BMP
  -------         PROC          MAIN
  -------         DO            
  D:0008H         SYMBOL        t
  -------         ENDDO         
  C:3E92H         LINE#         40
  C:3E92H         LINE#         41
  C:3E92H         LINE#         42
  C:3E95H         LINE#         45
  C:3E95H         LINE#         46
  C:3E95H         LINE#         48
  C:3E9AH         LINE#         49
  C:3E9DH         LINE#         50
  C:3EA5H         LINE#         51
  C:3EAEH         LINE#         52
  C:3EB7H         LINE#         53
  C:3EC0H         LINE#         54
  C:3EC9H         LINE#         55
  C:3ED2H         LINE#         56
  C:3EDBH         LINE#         58
  C:3EE8H         LINE#         59
  C:3EF5H         LINE#         60
  C:3F02H         LINE#         63
  C:3F16H         LINE#         66
  C:3F1DH         LINE#         67
  C:3F22H         LINE#         68
  C:3F36H         LINE#         70
  C:3F3DH         LINE#         71
  C:3F40H         LINE#         72
  C:3F47H         LINE#         73
  -------         ENDPROC       MAIN
  -------         ENDMOD        MAIN

  -------         MODULE        OLED
  C:0000H         SYMBOL        _ICE_DUMMY_
  B:0090H.2       PUBLIC        OLED_RST
  D:0090H         PUBLIC        P1
  C:42E4H         PUBLIC        OPEN_DC_POWER
  C:42CAH         PUBLIC        _Write_Parameter
  B:0090H.4       PUBLIC        OLED_CS
  C:4257H         PUBLIC        _Column_Address
  C:4294H         PUBLIC        _Set_Colume_Address
BL51 BANKED LINKER/LOCATER V6.22                                                      04/19/2018  15:18:06  PAGE 5


  C:417DH         PUBLIC        _OLED_ShowString
  C:3C0DH         PUBLIC        _OLED_ShowChar
  B:0090H.3       PUBLIC        OLED_RS
  C:3235H         PUBLIC        F6x8
  C:3A4DH         PUBLIC        Hzk
  C:42EEH         PUBLIC        OFF_DC_POWER
  B:0090H.1       PUBLIC        OLED_SDIN
  C:4273H         PUBLIC        _Write_Register
  C:41DFH         PUBLIC        _Write_IIC_Byte
  C:42C5H         PUBLIC        IIC_Wait_Ack
  C:345DH         PUBLIC        F8X16
  C:41FEH         PUBLIC        _ClearLED
  C:42F8H         PUBLIC        IIC_Start
  C:3F4AH         PUBLIC        Initial_ssd1327
  C:3D6EH         PUBLIC        _OLED_ShowCHinese
  C:41AEH         PUBLIC        Rainbow
  C:4108H         PUBLIC        _OLED_ShowNum
  C:4301H         PUBLIC        IIC_Stop
  C:423FH         PUBLIC        _oled_pow
  C:4281H         PUBLIC        _Row_Address
  B:0090H.0       PUBLIC        OLED_SCL
  C:4220H         PUBLIC        _Delay
  C:42A7H         PUBLIC        _Set_Row_Address
  C:408AH         PUBLIC        _OLED_DrawBMP
  -------         PROC          _DELAY
  D:0006H         SYMBOL        Data
  -------         DO            
  D:0004H         SYMBOL        temp
  -------         ENDDO         
  C:4220H         LINE#         40
  C:4220H         LINE#         41
  C:4220H         LINE#         43
  C:4229H         LINE#         44
  C:4229H         LINE#         45
  C:4237H         LINE#         46
  C:423EH         LINE#         47
  -------         ENDPROC       _DELAY
  -------         PROC          IIC_START
  C:42F8H         LINE#         48
  C:42F8H         LINE#         49
  C:42F8H         LINE#         51
  C:42FAH         LINE#         52
  C:42FCH         LINE#         53
  C:42FEH         LINE#         54
  C:4300H         LINE#         55
  -------         ENDPROC       IIC_START
  -------         PROC          IIC_STOP
  C:4301H         LINE#         60
  C:4301H         LINE#         61
  C:4301H         LINE#         62
  C:4303H         LINE#         64
  C:4305H         LINE#         65
  C:4307H         LINE#         67
  -------         ENDPROC       IIC_STOP
  -------         PROC          L?0114
  -------         ENDPROC       L?0114
  -------         PROC          IIC_WAIT_ACK
BL51 BANKED LINKER/LOCATER V6.22                                                      04/19/2018  15:18:06  PAGE 6


  C:42C5H         LINE#         69
  C:42C5H         LINE#         70
  C:42C5H         LINE#         88
  C:42C7H         LINE#         89
  C:42C9H         LINE#         90
  -------         ENDPROC       IIC_WAIT_ACK
  -------         PROC          L?0117
  -------         ENDPROC       L?0117
  -------         PROC          _WRITE_IIC_BYTE
  D:0007H         SYMBOL        IIC_Byte
  -------         DO            
  D:0006H         SYMBOL        i
  D:0005H         SYMBOL        m
  D:0007H         SYMBOL        da
  -------         ENDDO         
  C:41DFH         LINE#         95
  C:41DFH         LINE#         96
  C:41DFH         LINE#         99
  C:41DFH         LINE#         100
  C:41E1H         LINE#         101
  C:41E3H         LINE#         102
  C:41E3H         LINE#         103
  C:41E5H         LINE#         105
  C:41E8H         LINE#         106
  C:41EBH         LINE#         107
  C:41EFH         LINE#         108
  C:41F1H         LINE#         109
  C:41F5H         LINE#         110
  C:41F7H         LINE#         111
  C:41F9H         LINE#         112
  C:41FDH         LINE#         115
  -------         ENDPROC       _WRITE_IIC_BYTE
  C:426EH         SYMBOL        L?0116
  -------         PROC          L?0115
  -------         ENDPROC       L?0115
  C:426EH         SYMBOL        L?0116
  -------         PROC          _WRITE_REGISTER
  D:0004H         SYMBOL        Data
  C:4273H         LINE#         118
  C:4273H         LINE#         119
  C:4273H         LINE#         120
  C:4273H         LINE#         121
  C:4276H         LINE#         122
  C:4279H         LINE#         123
  C:427BH         LINE#         124
  C:427BH         LINE#         125
  C:427BH         LINE#         126
  C:427EH         LINE#         127
  -------         ENDPROC       _WRITE_REGISTER
  -------         PROC          _WRITE_PARAMETER
  D:0004H         SYMBOL        Data
  C:42CAH         LINE#         130
  C:42CAH         LINE#         131
  C:42CAH         LINE#         132
  C:42CAH         LINE#         133
  C:42CDH         LINE#         134
  C:42D0H         LINE#         135
BL51 BANKED LINKER/LOCATER V6.22                                                      04/19/2018  15:18:06  PAGE 7


  C:42D2H         LINE#         136
  C:42D2H         LINE#         137
  C:42D2H         LINE#         138
  C:42D5H         LINE#         139
  -------         ENDPROC       _WRITE_PARAMETER
  -------         PROC          _COLUMN_ADDRESS
  D:0002H         SYMBOL        a
  D:0003H         SYMBOL        b
  C:4257H         LINE#         149
  C:425BH         LINE#         150
  C:425BH         LINE#         151
  C:4260H         LINE#         152
  C:4267H         LINE#         153
  -------         ENDPROC       _COLUMN_ADDRESS
  -------         PROC          _ROW_ADDRESS
  D:0002H         SYMBOL        a
  D:0003H         SYMBOL        b
  C:4281H         LINE#         162
  C:4285H         LINE#         163
  C:4285H         LINE#         164
  C:428AH         LINE#         165
  C:428FH         LINE#         166
  -------         ENDPROC       _ROW_ADDRESS
  -------         PROC          _CLEARLED
  D:0009H         SYMBOL        color
  -------         DO            
  D:0003H         SYMBOL        j
  D:0002H         SYMBOL        i
  -------         ENDDO         
  C:41FEH         LINE#         174
  C:4200H         LINE#         175
  C:4200H         LINE#         178
  C:4207H         LINE#         180
  C:420EH         LINE#         181
  C:4210H         LINE#         182
  C:4210H         LINE#         183
  C:4212H         LINE#         184
  C:4212H         LINE#         185
  C:4217H         LINE#         186
  C:421BH         LINE#         187
  C:421FH         LINE#         188
  -------         ENDPROC       _CLEARLED
  -------         PROC          RAINBOW
  -------         DO            
  D:0003H         SYMBOL        j
  D:0002H         SYMBOL        i
  -------         ENDDO         
  C:41AEH         LINE#         189
  C:41AEH         LINE#         190
  C:41AEH         LINE#         193
  C:41B5H         LINE#         195
  C:41BCH         LINE#         196
  C:41BEH         LINE#         197
  C:41BEH         LINE#         198
  C:41C0H         LINE#         199
  C:41C0H         LINE#         200
  C:41CFH         LINE#         201
BL51 BANKED LINKER/LOCATER V6.22                                                      04/19/2018  15:18:06  PAGE 8


  C:41D3H         LINE#         202
  C:41D7H         LINE#         203
  -------         ENDPROC       RAINBOW
  -------         PROC          _SET_COLUME_ADDRESS
  D:0002H         SYMBOL        Addr1
  D:0003H         SYMBOL        Addr2
  C:4294H         LINE#         205
  C:4298H         LINE#         206
  C:4298H         LINE#         207
  C:429DH         LINE#         208
  C:42A2H         LINE#         209
  -------         ENDPROC       _SET_COLUME_ADDRESS
  -------         PROC          _SET_ROW_ADDRESS
  D:0002H         SYMBOL        Addr1
  D:0003H         SYMBOL        Addr2
  C:42A7H         LINE#         213
  C:42ABH         LINE#         214
  C:42ABH         LINE#         215
  C:42B0H         LINE#         216
  C:42B5H         LINE#         217
  -------         ENDPROC       _SET_ROW_ADDRESS
  -------         PROC          _OLED_SHOWCHAR
  D:000FH         SYMBOL        x
  D:0010H         SYMBOL        y
  D:0003H         SYMBOL        chr
  -------         DO            
  D:0011H         SYMBOL        c
  D:0001H         SYMBOL        i
  D:0003H         SYMBOL        j
  D:0012H         SYMBOL        Data1
  D:0013H         SYMBOL        Data2
  D:0014H         SYMBOL        DATA1
  -------         ENDDO         
  C:3C0DH         LINE#         221
  C:3C11H         LINE#         222
  C:3C15H         LINE#         225
  C:3C17H         LINE#         226
  C:3C1CH         LINE#         227
  C:3C24H         LINE#         229
  C:3C2EH         LINE#         231
  C:3C30H         LINE#         232
  C:3C30H         LINE#         233
  C:3C52H         LINE#         234
  C:3C74H         LINE#         235
  C:3C76H         LINE#         236
  C:3C76H         LINE#         237
  C:3C8CH         LINE#         238
  C:3C8CH         LINE#         239
  C:3C8FH         LINE#         240
  C:3C91H         LINE#         241
  C:3C94H         LINE#         242
  C:3CAAH         LINE#         243
  C:3CAAH         LINE#         244
  C:3CADH         LINE#         245
  C:3CADH         LINE#         246
  C:3CB2H         LINE#         247
  C:3CB5H         LINE#         248
BL51 BANKED LINKER/LOCATER V6.22                                                      04/19/2018  15:18:06  PAGE 9


  C:3CB9H         LINE#         249
  C:3CC2H         LINE#         253
  C:3CCCH         LINE#         254
  C:3CD9H         LINE#         255
  C:3CDBH         LINE#         256
  C:3CDBH         LINE#         257
  C:3CFDH         LINE#         258
  C:3D1FH         LINE#         259
  C:3D21H         LINE#         260
  C:3D21H         LINE#         261
  C:3D37H         LINE#         262
  C:3D37H         LINE#         263
  C:3D3AH         LINE#         264
  C:3D3CH         LINE#         265
  C:3D3FH         LINE#         266
  C:3D55H         LINE#         267
  C:3D55H         LINE#         268
  C:3D58H         LINE#         269
  C:3D58H         LINE#         270
  C:3D5DH         LINE#         271
  C:3D60H         LINE#         272
  C:3D64H         LINE#         273
  C:3D6DH         LINE#         274
  -------         ENDPROC       _OLED_SHOWCHAR
  -------         PROC          _OLED_SHOWSTRING
  D:0009H         SYMBOL        x
  D:000AH         SYMBOL        y
  D:000BH         SYMBOL        chr
  -------         DO            
  D:000EH         SYMBOL        j
  -------         ENDDO         
  C:417DH         LINE#         277
  C:4187H         LINE#         278
  C:4187H         LINE#         279
  C:418AH         LINE#         280
  C:419CH         LINE#         281
  C:41A3H         LINE#         282
  C:41A9H         LINE#         284
  C:41ABH         LINE#         285
  C:41ADH         LINE#         286
  -------         ENDPROC       _OLED_SHOWSTRING
  -------         PROC          _OLED_POW
  D:001EH         SYMBOL        m
  D:0001H         SYMBOL        n
  -------         DO            
  D:0006H         SYMBOL        result
  -------         ENDDO         
  C:423FH         LINE#         289
  C:4243H         LINE#         290
  C:4243H         LINE#         291
  C:4247H         LINE#         292
  C:4256H         LINE#         293
  C:4256H         LINE#         294
  -------         ENDPROC       _OLED_POW
  -------         PROC          _OLED_SHOWNUM
  D:0015H         SYMBOL        x
  D:0016H         SYMBOL        y
BL51 BANKED LINKER/LOCATER V6.22                                                      04/19/2018  15:18:06  PAGE 10


  D:0017H         SYMBOL        num
  D:0019H         SYMBOL        len
  D:001AH         SYMBOL        size
  -------         DO            
  D:001BH         SYMBOL        t
  D:001CH         SYMBOL        temp
  D:001DH         SYMBOL        enshow
  -------         ENDDO         
  C:4108H         LINE#         301
  C:4110H         LINE#         302
  C:4110H         LINE#         304
  C:4113H         LINE#         305
  C:411CH         LINE#         306
  C:411CH         LINE#         307
  C:413EH         LINE#         308
  C:414CH         LINE#         309
  C:414CH         LINE#         310
  C:4150H         LINE#         311
  C:4150H         LINE#         312
  C:4160H         LINE#         313
  C:4162H         LINE#         314
  C:4165H         LINE#         316
  C:4165H         LINE#         317
  C:4178H         LINE#         318
  C:417CH         LINE#         319
  -------         ENDPROC       _OLED_SHOWNUM
  -------         PROC          _OLED_SHOWCHINESE
  D:0009H         SYMBOL        x
  D:000AH         SYMBOL        y
  D:000BH         SYMBOL        no
  -------         DO            
  D:0001H         SYMBOL        i
  D:000CH         SYMBOL        j
  D:000DH         SYMBOL        Data1
  D:000EH         SYMBOL        Data2
  D:000FH         SYMBOL        DATA1
  -------         ENDDO         
  C:3D6EH         LINE#         322
  C:3D74H         LINE#         323
  C:3D76H         LINE#         326
  C:3D78H         LINE#         328
  C:3D80H         LINE#         330
  C:3D8AH         LINE#         332
  C:3D8DH         LINE#         333
  C:3D8DH         LINE#         334
  C:3DA9H         LINE#         335
  C:3DC5H         LINE#         336
  C:3DC7H         LINE#         337
  C:3DC7H         LINE#         338
  C:3DDDH         LINE#         339
  C:3DDDH         LINE#         340
  C:3DE0H         LINE#         341
  C:3DE2H         LINE#         342
  C:3DE5H         LINE#         343
  C:3DEAH         LINE#         344
  C:3DEAH         LINE#         345
  C:3DEDH         LINE#         346
BL51 BANKED LINKER/LOCATER V6.22                                                      04/19/2018  15:18:06  PAGE 11


  C:3DEDH         LINE#         347
  C:3DF2H         LINE#         348
  C:3DF5H         LINE#         349
  C:3DF9H         LINE#         350
  C:3E02H         LINE#         354
  C:3E0CH         LINE#         355
  C:3E19H         LINE#         357
  C:3E1CH         LINE#         358
  C:3E1CH         LINE#         359
  C:3E38H         LINE#         360
  C:3E54H         LINE#         361
  C:3E56H         LINE#         362
  C:3E56H         LINE#         363
  C:3E6CH         LINE#         364
  C:3E6CH         LINE#         365
  C:3E6FH         LINE#         366
  C:3E71H         LINE#         367
  C:3E74H         LINE#         368
  C:3E79H         LINE#         369
  C:3E79H         LINE#         370
  C:3E7CH         LINE#         371
  C:3E7CH         LINE#         372
  C:3E81H         LINE#         373
  C:3E84H         LINE#         374
  C:3E88H         LINE#         375
  C:3E91H         LINE#         376
  -------         ENDPROC       _OLED_SHOWCHINESE
  -------         PROC          _OLED_DRAWBMP
  D:0009H         SYMBOL        x1
  D:000AH         SYMBOL        y1
  D:000BH         SYMBOL        x2
  D:000CH         SYMBOL        y2
  D:000DH         SYMBOL        BMP
  -------         DO            
  D:0010H         SYMBOL        i
  D:0011H         SYMBOL        m
  D:0012H         SYMBOL        k
  -------         ENDDO         
  C:408AH         LINE#         378
  C:4090H         LINE#         379
  C:4090H         LINE#         380
  C:4093H         LINE#         381
  C:4097H         LINE#         383
  C:409CH         LINE#         385
  C:40A3H         LINE#         387
  C:40C3H         LINE#         388
  C:40C3H         LINE#         389
  C:40E3H         LINE#         390
  C:40E3H         LINE#         392
  C:40FFH         LINE#         394
  C:4103H         LINE#         396
  C:4107H         LINE#         397
  -------         ENDPROC       _OLED_DRAWBMP
  -------         PROC          OPEN_DC_POWER
  C:42E4H         LINE#         399
  C:42E4H         LINE#         400
  C:42E4H         LINE#         401
BL51 BANKED LINKER/LOCATER V6.22                                                      04/19/2018  15:18:06  PAGE 12


  C:42E6H         LINE#         402
  C:42E9H         LINE#         403
  -------         ENDPROC       OPEN_DC_POWER
  -------         PROC          OFF_DC_POWER
  C:42EEH         LINE#         405
  C:42EEH         LINE#         406
  C:42EEH         LINE#         407
  C:42F0H         LINE#         408
  C:42F3H         LINE#         409
  -------         ENDPROC       OFF_DC_POWER
  -------         PROC          INITIAL_SSD1327
  C:3F4AH         LINE#         411
  C:3F4AH         LINE#         412
  C:3F4AH         LINE#         413
  C:3F4CH         LINE#         414
  C:3F4EH         LINE#         415
  C:3F50H         LINE#         416
  C:3F57H         LINE#         417
  C:3F59H         LINE#         419
  C:3F5EH         LINE#         420
  C:3F63H         LINE#         421
  C:3F68H         LINE#         422
  C:3F6DH         LINE#         423
  C:3F72H         LINE#         424
  C:3F77H         LINE#         425
  C:3F7CH         LINE#         426
  C:3F81H         LINE#         427
  C:3F86H         LINE#         428
  C:3F8BH         LINE#         429
  C:3F90H         LINE#         430
  C:3F95H         LINE#         431
  C:3F9AH         LINE#         432
  C:3F9FH         LINE#         433
  C:3FA4H         LINE#         434
  C:3FA9H         LINE#         435
  C:3FAEH         LINE#         436
  C:3FB3H         LINE#         437
  C:3FB5H         LINE#         438
  C:3FB8H         LINE#         439
  C:3FBDH         LINE#         440
  C:3FC2H         LINE#         441
  C:3FC7H         LINE#         442
  C:3FCCH         LINE#         443
  C:3FD1H         LINE#         444
  C:3FD6H         LINE#         445
  C:3FDBH         LINE#         446
  C:3FE0H         LINE#         447
  C:3FE5H         LINE#         448
  -------         ENDPROC       INITIAL_SSD1327
  -------         ENDMOD        OLED

  -------         MODULE        ?C?CLDOPTR
  C:3FEAH         PUBLIC        ?C?CLDOPTR
  -------         ENDMOD        ?C?CLDOPTR

  -------         MODULE        ?C?IMUL
  C:4017H         PUBLIC        ?C?IMUL
BL51 BANKED LINKER/LOCATER V6.22                                                      04/19/2018  15:18:06  PAGE 13


  -------         ENDMOD        ?C?IMUL

  -------         MODULE        ?C?UIDIV
  C:4029H         PUBLIC        ?C?UIDIV
  -------         ENDMOD        ?C?UIDIV

  -------         MODULE        ?C?OFFXADD
  C:407EH         PUBLIC        ?C?OFFXADD
  -------         ENDMOD        ?C?OFFXADD

*** WARNING L16: UNCALLED SEGMENT, IGNORED FOR OVERLAY PROCESS
    SEGMENT: ?PR?_COLUMN_ADDRESS?OLED

*** WARNING L16: UNCALLED SEGMENT, IGNORED FOR OVERLAY PROCESS
    SEGMENT: ?PR?_ROW_ADDRESS?OLED

*** WARNING L16: UNCALLED SEGMENT, IGNORED FOR OVERLAY PROCESS
    SEGMENT: ?PR?_OLED_SHOWNUM?OLED

*** WARNING L16: UNCALLED SEGMENT, IGNORED FOR OVERLAY PROCESS
    SEGMENT: ?PR?OFF_DC_POWER?OLED

Program Size: data=32.0 xdata=0 code=17160
LINK/LOCATE RUN COMPLETE.  4 WARNING(S),  0 ERROR(S)
